:100000003BC071C154C053C052C051C050C04FC05A
:100010004EC04DC04CC04BC04AC049C048C047C08C
:1000200046C045C044C004030904180372006100BF
:10003000700068006E00650074002E006E006500A0
:1000400074001203550053004200540065006E0016
:100050006B00690012010101FF0000088117980A76
:1000600008010102030109021200010100803209A6
:10007000040000000000000011241FBECFE5D4E002
:10008000DEBFCDBF11E0A0E6B0E0EAE7FBE102C0D1
:1000900005900D92A238B107D9F711E0A2E8B1E0BE
:1000A00001C01D92AD3CB107E1F791D364CDA8CF5B
:1000B00082E891E08093AE010B968093AD0185B705
:1000C000836085BF8BB780648BBF08950F931F93A8
:1000D000CF93DF938091B301882309F49BC0482F0D
:1000E000435047FD95C022E831E09091AD019F5FFC
:1000F0008091B0018D3209F083C0483009F080C092
:10010000C92FD32F8881807609F06BC01092AB0184
:100110008981882359F41092AC018BEA91E0909385
:10012000B2018093B10120E892E063C0853021F4F0
:100130008A818093B4014AC08630D9F58B818130A1
:1001400019F484E590E023C0823019F486E690E04B
:100150001EC0833009F04BC08A81882349F486E2AF
:1001600090E09093B2018093B10120EC94E041C003
:10017000813049F48AE290E09093B2018093B1011A
:1001800020EC98E136C0823049F482E490E090930C
:10019000B2018093B10120EC92E12BC0833039F59C
:1001A00082E690E09093B2018093B10120E89EE056
:1001B00020C0883019F486EB91E00CC0893021F41E
:1001C0008A818093B60102C08A3011F020E810C005
:1001D0008BEA91E09093B2018093B10120E891E025
:1001E00008C0892F932F37D3982F20E802C020EC26
:1001F00090E08F81882339F48E81891728F003C01D
:1002000020E880E001C0892F20939801809360004E
:100210001092B301909160009F3F09F448C0809113
:10022000610084FF44C0192F993008F018E0911B39
:10023000909360008091980180FD02C00BE401C0A2
:1002400003EC8F5F809398012091B1013091B2014E
:1002500086FD05C0D901912FE3EAF1E011C0A3EAC0
:10026000B1E080E090E006C0F901E80FF91FE491E9
:10027000ED9301961817C1F705C08D9181939150A8
:100280009923D9F7F901E10FF11DF093B201E09341
:10029000B10183EA91E0612FC9D1183019F08FEFD5
:1002A000809360000093A2011C5F1093610080B3F3
:1002B000857019F01092990111C0809199018823DD
:1002C00069F494E680B3857049F49150D9F781E0E0
:1002D000809399011092B4011092AF01DF91CF91F8
:1002E0001F910F9108950F930FB70F93809BFECF2F
:1002F000809B06C0809B04C0809B02C0000000C0A1
:100300001F933F932F9331E014E000B3102710FDAB
:1003100032E0102F3A95C9F700FDE3C000B3102773
:1003200020E010FB20F9DF9310B3012700FB21F937
:10033000CF93C091AE0100B3102710FB22F93BE030
:10034000D1E04F9310B3012700FB23F94FEF0000DA
:1003500055C0809BFECF809B06C0809B04C0809BC5
:1003600002C0000000C0DF9100C0CDCF10B31570F7
:1003700079F14F7D206213C000B3057049F14F7BC6
:10038000206415C0057021F1102F206800B319C03A
:1003900000B30570E9F04E7F216018C039F300B357
:1003A0000570B1F0102710FB26F9223028F310B3A6
:1003B000012700FB27F9422749934FEF00B3243070
:1003C00008F3102710FB20F9297F11F310B31570E3
:1003D000E1F1012700FB21F9237FF1F000B3057063
:1003E000A1F1102710FB22F9277EE1F010B30127BD
:1003F00000FB23F93A9541F12F7CD1F000B3057051
:1004000021F1102710FB24F92F79C1F010B3012737
:1004100000FB25F92F73C2CF10B31570B1F04D7FDB
:100420002260DCCF00B3057081F04B7F2460DECF0B
:1004300010B3157051F0477F2860E0CF00B305700E
:1004400021F04F7E2061E2CF3BC03C2FC091AE0136
:100450003C1B00E433300ABF98F108811981412F19
:100460001F772091AF010D3279F1013E69F1093614
:10047000C1F00777033421F51091B501112301F183
:100480000091B3010030C1F53430C2F13093B301B3
:100490001093B0010091AD01C093AD010093AE0186
:1004A0002DC0121769F43091610034FD23C00AE5B4
:1004B00000936100C2EAD1E025C000270093B50196
:1004C0004F91CF91DF910DC01217B9F70093B5018D
:1004D0000AE5009361004F91CF910AB706FD39CF2D
:1004E000DF9100E40ABF2F913F911F910F910FBF41
:1004F0000F911895432F03C04AE501C042EDC4E1B6
:10050000D0E032E05F9355E0909A02B3889A8A9ADD
:1005100020E80FC0052710E002BB10C0052710E03F
:10052000089402BB13C0052710E015C0052710E092
:1005300019C020FF052702BB279517951C3F50F7D0
:1005400020FF0527279502BB17951C3F38F720FF92
:1005500005272795179502BB1C3F28F720FF052785
:10056000279517951C3F02BB08F700C0499120FF53
:10057000052702BB279517951C3F80F520FF05270F
:10058000279502BB17951C3F68F520FF0527279587
:10059000179502BB1C3F58F520FF05272795179597
:1005A0001C3F02BB38F5242F3A9519F60A7F5F915C
:1005B00002BB32E03A95F1F71091B401C651D04038
:1005C00011F01093AF01016011B31A7F02BB0A7FD3
:1005D0004F91CF9111BB02BBDF9183CF052710E074
:1005E00002BBCACF052710E0089402BBCDCF052778
:1005F00010E0CFCF052710E0D3CFA82FB92F8FEF72
:100600009FEF41E050EA615070F02D9138E0722F79
:10061000782796958795269570FF02C084279527A1
:100620003A95A9F7F0CF809590950895E6DF8D93E0
:100630009D930895FC0197FD06C08630910518F43E
:10064000E954FE4F67830895E4E6F0E08091BE012F
:1006500080936400109265008091BF0180936600D2
:1006600013828091C0018093680015828091C1013E
:1006700080936A0017828091C20180936C0011867A
:100680008091C30180936E00138608959AD1E4E6A9
:10069000F0E08091BE01809364001092650080912B
:1006A000BF018093660013828091C001809368002F
:1006B00015828091C10180936A0017828091C201E6
:1006C00080936C0011868091C30180936E00138625
:1006D0000895892B19F085B3806302C085B38F7CA0
:1006E00085BB60B981B18C7F81B908950F931F9349
:1006F000982FFA01D8016115710531F421153105E2
:1007000079F52FEF3FEF5FC084EA86BF06B607FE9C
:10071000FDCF81B1887F883019F021E030E053C0EF
:10072000892F880F83B984E886BF06B607FEFDCF00
:1007300081B1887F883109F042C008C0808183B9C7
:1007400046BF06B607FEFDCF319601C044E86150B2
:1007500070408FEF6F3F780789F72115310551F110
:1007600084EA86BF06B607FEFDCF81B1803119F05D
:1007700023E030E026C0990F916093B984E886BFEA
:1007800006B607FEFDCF81B1803479F024E030E079
:1007900018C02150304011F096BF01C046BF06B6C8
:1007A00007FEFDCF83B18D9302C044E894EC211580
:1007B000310579F784E986BF20E030E004C022E00B
:1007C00030E084E986BFC9011F910F9108952EE0A2
:1007D00088E190E00FB6F894A89581BD0FBE21BDC9
:1007E0008FEF88BB87BB85BB14BA24D1F2D02CDF36
:1007F00088EF82BB85E081BB81B38A7F81BB58DCF7
:10080000789414D3892B09F0FFCFA8955FDCFDCF36
:10081000EF92FF920F931F93CF93DF936AE070E004
:10082000F0D8EB0100E010E080E3E82E85E7F82E39
:1008300007C0A8954BDCC7010197F1F70F5F1F4F69
:100840000C171D07B4F342DCDF91CF911F910F917C
:10085000FF90EF9008951F93CF93DF93EC011092D8
:100860007000C1D2AC019C01285F3F4F6AE971E082
:100870007093B2016093B1011981103199F0113177
:1008800038F4113009F44AC0123009F094C065C040
:10089000113F09F47AC0123F09F482C0103F09F0F9
:1008A0008AC065C08A8190E0821793070CF083C0EC
:1008B00010939A012A81822F90E08417950774F093
:1008C000822F841B65E070E04AE050E0BED0909338
:1008D0009B0180939C0122E030E00CC0822F6F5F6F
:1008E0007F4F92D29C0197FF05C010929A0181E040
:1008F00090E063C0D901119690E0EAE9F1E0AD0122
:100900004E0F5F1F02C081919827E417F507D9F7B2
:10091000A656BE4F9C93C90102964FC08A8190E0B3
:10092000821793070CF047C010939A018A81E82F31
:10093000F0E0E417F50734F0E41BF50BE954FE4F43
:10094000858501C053D280939B0180919B0190913A
:100950009A01892780939C0107C010939A012093E4
:100960009B01122710939C0183E090E026C08A81AE
:100970008F3F11F48BDE03C090E06B815BDE80EF74
:1009800080939A0180939B0113C08A81E82FF0E045
:10099000E830F10584F4E954FE4F8B81858703C06C
:1009A0008A818093CC010DD010939A0110939B0102
:1009B00082E090E002C080E090E0DF91CF911F9153
:1009C000089587EB91E060E070E046E150E0BDD82B
:1009D000089587EB91E060E070E046E150E0A5D833
:1009E00087EB91E061E770E047E050E08AD800973C
:1009F00001F1A7EBB1E0E1E7F0E087E001900D92B3
:100A00008150E1F78EEB91E06FE370E046E050E05B
:100A100085D884EC91E06FEF70E048E050E07ED83C
:100A20001092CC0187EB91E060E070E046E150E08D
:100A30008CD808958091CC01882319F480E487B97B
:100A400001C017B887E886B908952F923F924F9258
:100A50005F926F927F928F929F92AF92BF92CF924E
:100A6000DF92EF92FF920F931F93DF93CF93CDB757
:100A7000DEB728970FB6F894DEBF0FBECDBF982F14
:100A80007A836983803118F02FEF3FEF85C0809122
:100A9000CC01882319F4906497B905C0892F992750
:100AA00087FD909587B918861F82662477244301B5
:100AB00022243324CA01AA2797FDA095BA2F8B833D
:100AC0009C83AD83BE8357C0369A349BFECF84B1DE
:100AD000A82FB0E085B1582E4424A429B529B887A1
:100AE000AF836B817C818D819E81EBD45B016C0136
:100AF00020E030E84BE355E46ED37B018C0120E02D
:100B000030E040E85FE3B2D488231CF461E070E099
:100B10001FC0C801B70120E03FEF4FE757E450D4B2
:100B200018169CF4C601B50120E030E040E251E423
:100B300052D38DD106C08CE291E00197F1F761505C
:100B4000704061157105B9F706C0C801B7017FD1C2
:100B5000CB010197F1F78F81988526E0880F991FC7
:100B60002A95E1F7A0E0B0E0680E791E8A1E9B1E70
:100B70000894211C311CA981BA812A163B060CF469
:100B8000A3CFA130B10551F09D01442737FD409519
:100B9000542FC401B30148D738872F838F8198859C
:100BA00028960FB6F894DEBF0FBECDBFCF91DF9170
:100BB0001F910F91FF90EF90DF90CF90BF90AF907B
:100BC0009F908F907F906F905F904F903F902F906D
:100BD0000895000000000000000000000000000078
:100BE0000000000000000000000000000000000005
:100BF00000000000000000000000000000000000F5
:100C000000000000000000000000000000000000E4
:100C100000000000000000000000000000000000D4
:100C200000000000000000000000000000000000C4
:100C300000000000000000000000000000000000B4
:100C400000000000000000000000000000000000A4
:100C50000000000000000000000000000000000094
:100C60000000000000000000000000000000000084
:100C70000000000000000000000000000000000074
:100C80000000000000000000000000000000000064
:100C900000000895A39AAB98A298AA9A08950F937A
:100CA0001F93082FAB9A95DFAA98A29A92DFAB9870
:100CB00090DFAB9A8EDFA298AA9A8BDFAB9889DF80
:100CC00010E007FF03C0A298AA9A02C0AA98A29AAD
:100CD00080DFAB9A7EDFAB981F5F183011F0000FFA
:100CE000F0CFA298AA9A75DFAB9A73DF83B3AB9863
:100CF00082FF03C02FEF3FEF04C09A9BFECF20E09E
:100D000030E0C9011F910F9108950F931F93082F91
:100D100060DF10E007FF03C0A298AA9A02C0AA9859
:100D2000A29A57DFAB9A55DFAB9853DF1F5F18309D
:100D300011F0000FEFCFA298AA9A4BDFAB9A49DFD0
:100D400083B3AB9882FF03C02FEF3FEF04C09A9BA1
:100D5000FECF20E030E0C9011F910F910895EF927E
:100D6000FF920F931F93CF93DF937C01062F10E028
:100D7000C0E0D0E02EDFAB9A2CDF110F9A99116002
:100D8000AB982196C830D105A9F7F701108300234D
:100D900011F4AA98A29A1DDFAB9A1BDFAB98A29818
:100DA000AA9A17DF80E090E0DF91CF911F910F9119
:100DB000FF90EF900895CF93DF93EB0170DF892BC5
:100DC00019F02FEF3FEF0BC09A99FECFCE0160E0F4
:100DD000C6DFCE01019661E0C2DF20E030E0C9014C
:100DE000DF91CF91089582E090E00895882329F063
:100DF000813031F424E030E005C023E030E002C06F
:100E00002FEF3FEFC9010895882329F0813029F0A1
:100E10002FEF3FEF09C083E001C085E0CCDF9C01EC
:100E2000009711F422E030E0C901089584EF91E0C9
:100E30002CE231E0F9013197F1F70197D9F72ADF78
:100E400086E02DDF80E061DF80E090E00895EF92A2
:100E5000FF920F931F937B018C0120E030E040E074
:100E60005FE4D9D288237CF0C801B70120E030E0EC
:100E700040E05FE45ED17FD39B01AC012050304065
:100E80004040504805C0C801B70175D39B01AC0173
:100E9000B901CA011F910F91FF90EF900895A0E052
:100EA000B0E0E4E5F7E0F6C5DC012B01FA019C9126
:100EB000923008F439C1EB018881823008F433C1E3
:100EC000943069F4843009F02FC111969C911197E8
:100ED0008981981709F428C1AAE7B0E025C18430B8
:100EE00009F421C18230A9F4923009F01DC19A01A0
:100EF000AD0188E0EA010990AE01E90109929E0185
:100F00008150C1F7E201898111969C9189238183E7
:100F100008C1923009F407C112962D903C901397A6
:100F2000EB018A819B811496AD90BD90CD90DC90B1
:100F30001797EC80FD800E811F819101281B390BD2
:100F4000B90137FF04C066277727621B730B603235
:100F500071050CF061C0121613066CF537014801DB
:100F6000062E04C096948794779467940A94D2F7D7
:100F700021E030E040E050E004C0220F331F441F66
:100F8000551F6A95D2F721503040404050402E21E5
:100F90003F2140235123211531054105510521F001
:100FA00021E030E040E050E079018A01E628F728AE
:100FB000082919293CC0232BD1F1260E371E3501F3
:100FC0004601062E04C096948794779467940A94F9
:100FD000D2F721E030E040E050E004C0220F331FA0
:100FE000441F551F6A95D2F7215030404040504071
:100FF0002A213B214C215D21211531054105510557
:1010000021F021E030E040E050E059016A01A628DB
:10101000B728C828D9280BC0821593052CF01C01CD
:10102000AA24BB24650103C0EE24FF248701119686
:101030009C91D20111968C91981709F445C099237F
:1010400039F0A80197012A193B094C095D0906C02E
:10105000A60195012E193F09400B510B57FD08C001
:1010600011823382228224833583468357831DC0B5
:1010700081E081833382228288279927DC01821BC9
:10108000930BA40BB50B84839583A683B7830DC004
:10109000220F331F441F551F2483358346835783F4
:1010A0008281938101979383828324813581468154
:1010B0005781DA01C9010197A109B1098F5F9F4FDB
:1010C000AF4FBF4328F30BC0918333822282EA0CD7
:1010D000FB1C0C1D1D1DE482F5820683178383E033
:1010E0008083248135814681578157FF1AC0C90109
:1010F000AA2797FDA095BA2F81709070A070B0704C
:101100005695479537952795822B932BA42BB52B76
:1011100084839583A683B783828193810196938389
:101120008283DF0101C0D201CD01CDB7DEB7E2E19C
:10113000CDC4A0E2B0E0EEE9F8E0B8C469837A83F8
:101140008B839C832D833E834F835887E9E0EE2E6B
:10115000F12CEC0EFD1ECE010196B70181D38E015C
:101160000F5E1F4FCE010596B8017AD38A8991E0B0
:1011700089278A8BC701B801AE01475E5F4F8FDEBA
:101180009AD2A096E6E0AEC4A0E2B0E0E9ECF8E0C6
:101190008DC469837A838B839C832D833E834F83A5
:1011A0005887F9E0EF2EF12CEC0EFD1ECE010196D2
:1011B000B70156D38E010F5E1F4FCE010596B801C1
:1011C0004FD3C701B801AE01475E5F4F68DE73D2EF
:1011D000A096E6E087C4A0E2B0E0E0EFF8E05AC4F1
:1011E00069837A838B839C832D833E834F835887C7
:1011F000CE010196BE01675F7F4F32D3CE010596C7
:10120000BE016F5E7F4F2CD39985923088F089891B
:101210008230C8F0943019F4823051F404C0843024
:1012200029F4923081F48AE790E0C6C0923049F404
:1012300020E09A858A89981321E02A87CE010996B1
:10124000BBC0823049F420E09A858A89981321E056
:101250002A8BCE014196B0C02D843E844F8458889D
:101260006D887E888F88988CEE24FF248701AA24BD
:10127000BB24650140E050E060E070E0E0E0F0E0B9
:10128000C10181709070892BE9F0E60CF71C081DF4
:10129000191D9A01AB012A0D3B1D4C1D5D1D80E0FF
:1012A00090E0A0E0B0E0E614F7040805190520F48A
:1012B00081E090E0A0E0B0E0BA01A901480F591F19
:1012C0006A1F7B1FAA0CBB1CCC1CDD1C97FE08C030
:1012D00081E090E0A0E0B0E0A82AB92ACA2ADB2A7F
:1012E0003196E032F10549F0660C771C881C991C98
:1012F0005694479437942794C3CFFA85EA892B896B
:101300003C898B859C85280F391F2E5F3F4F17C066
:10131000CA0181709070892B61F016950795F7943A
:10132000E79480E090E0A0E0B0E8E82AF92A0A2BF0
:101330001B2B76956795579547952F5F3F4F77FD08
:10134000E7CF0CC0440F551F661F771F17FD416084
:10135000EE0CFF1C001F111F21503040403090E068
:10136000590790E0690790E4790760F32B8F3C8F71
:10137000DB01CA018F779070A070B0708034910546
:10138000A105B10561F447FD0AC0E114F1040105AE
:10139000110529F0405C5F4F6F4F7F4F40781A8EE8
:1013A000FE1711F081E08A8F4D8F5E8F6F8F78A3CB
:1013B00083E0898FCE0149967ED1A096E2E186C373
:1013C000A8E1B0E0E5EEF9E071C369837A838B832D
:1013D0009C832D833E834F83588789E0E82EF12C30
:1013E000EC0EFD1ECE010196B7013AD28E010F5EC2
:1013F0001F4FCE010596B80133D28985823038F06F
:101400008989823020F0C701B801A2D201C08FEFD4
:101410006896E6E067C3A8E1B0E0E0E1FAE046C321
:1014200069837A838B839C832D833E834F83588784
:1014300089E0E82EF12CEC0EFD1ECE010196B701DD
:101440000FD28E010F5E1F4FCE010596B80108D254
:101450008985823038F08989823020F0C701B8014F
:1014600077D201C08FEF6896E6E03CC3A8E1B0E018
:10147000EBE3FAE01BC369837A838B839C832D8320
:101480003E834F83588789E0E82EF12CEC0EFD1E39
:10149000CE010196B701E4D18E010F5E1F4FCE0140
:1014A0000596B801DDD18985823038F0898982308E
:1014B00020F0C701B8014CD201C081E06896E6E097
:1014C00011C3A8E0B0E0E6E6FAE0EDC29B01AC0192
:1014D00083E08983DA01C9018827B7FD83959927BD
:1014E000AA27BB27B82E211531054105510519F44E
:1014F00082E0898339C08823A9F0203080E0380752
:1015000080E0480780E8580729F460E070E080E058
:101510009FEC2EC0EE24FF248701E21AF30A040B8D
:10152000150B02C079018A018EE1C82ED12CDC8214
:10153000CB82ED82FE820F831887C801B7016CD081
:1015400001971816190684F4082E04C0EE0CFF1C2F
:10155000001F111F0A94D2F7ED82FE820F831887B5
:10156000C81AD90ADC82CB82BA82CE010196A3D0F6
:101570002896E9E0B4C2ACE0B0E0E0ECFAE09AC250
:1015800069837A838B839C83CE010196BE016B5F56
:101590007F4F66D18D81823061F1823050F184308D
:1015A00021F48E81882351F12EC02F81388537FD9B
:1015B00020C06E812F3131051CF06623F9F023C065
:1015C0008EE190E0821B930B29853A854B855C85E3
:1015D00004C056954795379527958A95D2F7662387
:1015E000B1F050954095309521953F4F4F4F5F4F4B
:1015F0000EC020E030E040E050E009C02FEF3FEFA8
:101600004FEF5FE704C020E030E040E050E8B90170
:10161000CA012C96E2E06AC2EF92FF920F931F93E9
:101620007B018C0180E0E81680E0F80681E0080785
:1016300080E0180788F48FEFE816F1040105110522
:1016400031F028F088E090E0A0E0B0E017C080E042
:1016500090E0A0E0B0E012C080E0E81680E0F8067C
:1016600080E0080781E0180728F088E190E0A0E01A
:10167000B0E004C080E190E0A0E0B0E020E230E023
:1016800040E050E0281B390B4A0B5B0B04C0169559
:101690000795F794E7948A95D2F7F701EE57FF4F35
:1016A0008081281B310941095109C9011F910F91FE
:1016B000FF90EF900895DF92EF92FF920F931F93A8
:1016C000FC01E480F58006811781D1808081823021
:1016D00048F480E090E0A0E1B0E0E82AF92A0A2B83
:1016E0001B2BA5C0843009F49FC0823021F4EE2466
:1016F000FF24870105C0E114F1040105110519F467
:10170000E0E0F0E096C0628173819FEF6238790774
:101710000CF05BC022E83FEF261B370B2A31310566
:101720002CF020E030E040E050E02AC0B801A701F2
:10173000022E04C076956795579547950A94D2F77F
:1017400081E090E0A0E0B0E004C0880F991FAA1FDC
:10175000BB1F2A95D2F70197A109B1098E219F21BC
:10176000A023B1230097A105B10521F081E090E00D
:10177000A0E0B0E09A01AB01282B392B4A2B5B2B60
:10178000DA01C9018F779070A070B0708034910534
:10179000A105B10539F427FF09C0205C3F4F4F4F29
:1017A0005F4F04C0215C3F4F4F4F5F4FE0E0F0E0E0
:1017B0002030A0E03A07A0E04A07A0E45A0710F062
:1017C000E1E0F0E079018A0127C06038710564F535
:1017D000FB01E158FF4FD801C7018F779070A070CF
:1017E000B07080349105A105B10539F4E7FE0DC054
:1017F00080E490E0A0E0B0E004C08FE390E0A0E0DF
:10180000B0E0E80EF91E0A1F1B1F17FF05C0169552
:101810000795F794E794319687E016950795F79426
:10182000E7948A95D1F705C0EE24FF248701EFEFF6
:10183000F0E06E2F679566276795902F9F77D79476
:10184000DD24D7948E2F8695492F462B582F5D295E
:10185000B701CA011F910F91FF90EF90DF9008959B
:10186000FC01DB01408151812281622F6F7770E0A2
:10187000221F2227221F9381892F880F822B282F36
:1018800030E0991F9927991F11969C931197211564
:101890003105A9F5411551056105710511F482E085
:1018A00037C082E89FEF13969C938E9312979A010C
:1018B000AB0167E0220F331F441F551F6A95D1F714
:1018C00083E08C930DC0220F331F441F551F1296C7
:1018D0008D919C911397019713969C938E931297D9
:1018E000203080E0380780E0480780E4580758F34C
:1018F00014962D933D934D935C93179708952F3F26
:10190000310579F4411551056105710519F484E03B
:101910008C93089564FF03C081E08C9312C01C92E5
:1019200010C02F57304013963C932E93129783E0AC
:101930008C9387E0440F551F661F771F8A95D1F758
:10194000706414964D935D936D937C9317970895EF
:101950001F93DC01FB019C91923008F447C0808109
:10196000823008F443C0943051F411961C918430B5
:1019700099F58181682F70E0611B71093FC0843047
:1019800021F0923031F48230B9F18181882389F1DC
:101990002DC011961C9111978230F1F0818118179A
:1019A000D9F412962D913C911397828193818217DD
:1019B000930794F028173907BCF014968D919D91E8
:1019C0000D90BC91A02D2481358146815781281727
:1019D00039074A075B0718F4112341F00AC0821740
:1019E0009307A407B50740F4112319F061E070E0F4
:1019F00005C06FEF7FEF02C060E070E0CB011F9188
:101A0000089597FB092E07260AD077FD04D02ED023
:101A100006D000201AF4709561957F4F0895F6F76F
:101A2000909581959F4F0895A1E21A2EAA1BBB1B8A
:101A3000FD010DC0AA1FBB1FEE1FFF1FA217B3079A
:101A4000E407F50720F0A21BB30BE40BF50B661FB0
:101A5000771F881F991F1A9469F760957095809574
:101A600090959B01AC01BD01CF010895AA1BBB1B42
:101A700051E107C0AA1FBB1FA617B70710F0A61B8E
:101A8000B70B881F991F5A95A9F780959095BC01AF
:101A9000CD0108952F923F924F925F926F927F9265
:101AA0008F929F92AF92BF92CF92DF92EF92FF926E
:101AB0000F931F93CF93DF93CDB7DEB7CA1BDB0B1A
:101AC0000FB6F894DEBF0FBECDBF09942A883988BF
:101AD00048885F846E847D848C849B84AA84B984C6
:101AE000C884DF80EE80FD800C811B81AA81B981D2
:101AF000CE0FD11D0FB6F894DEBF0FBECDBFED01E6
:101B00000895FB01DC0104C08D910190801921F43E
:101B100041505040C8F7881B990B0895DC0101C063
:101B20006D9341505040E0F70895DC01CB01FC017A
:101B3000E199FECF06C0FFBBEEBBE09A31960DB235
:101B40000D9241505040B8F70895DC01CB0102C01E
:101B50002D9105D041505040D8F70895262FE19996
:101B6000FECF9FBB8EBB2DBB0FB6F894E29AE19AD5
:0A1B70000FBE01960895F894FFCF10
:101B7A00FF5A0E034100420043004400450046005C
:101B8A000154656E6B694366310000000000000075
:101B9A000000000102020303030304040404040412
:101BAA0004040505050505050505050505050505DD
:101BBA0005050606060606060606060606060606BD
:101BCA0006060606060606060606060606060606AB
:101BDA00060607070707070707070707070707078D
:101BEA00070707070707070707070707070707077B
:101BFA00070707070707070707070707070707076B
:101C0A00070707070707070707070707070707075A
:101C1A00070708080808080808080808080808083C
:101C2A00080808080808080808080808080808082A
:101C3A00080808080808080808080808080808081A
:101C4A00080808080808080808080808080808080A
:101C5A0008080808080808080808080808080808FA
:101C6A0008080808080808080808080808080808EA
:101C7A0008080808080808080808080808080808DA
:101C8A0008080808080808080808080808080808CA
:021C9A00080838
:00000001FF
